:020000040000FA
:100000008E018F0190019101023092000130930026
:1000100094018501860183168501803086000430B5
:1000200081008312861FCE28372071200B1D1628D1
:100030008B01A0200C08143A031D222830308600C2
:100040001F3085008C0B162814280F398207403486
:10005000793424343034193412340234783400348E
:1000600010347F347F347F347F347F347F346D307D
:100070008C008E0A0E08093C031808006F308C00B3
:100080008E018F0A0F08053C0318080071308C00A0
:100090008F01900A1008093C0318080073308C0087
:1000A0009001910A1108053C0318080072308C0079
:1000B00091011308013C03186728920A1208033CB7
:1000C000031808006F308C00920193010800920A17
:1000D0001208093C031808006E308C009201930A44
:1000E00008009501940A1408083C031C94011408A4
:1000F000013A03198928033A03198E28013A031992
:100100009128073A03199428303086001F30850063
:10011000080095151308031D9628080015151208E8
:100120009628951411089628151410089700252074
:100130008D001F3985000D0C30391504860008002C
:10014000861B0800950803190800970A1708093C40
:10015000031C970117089620C620861FAD28C620CD
:10016000861FAD2814309600861FA528C620960B42
:10017000B428170894018F018E0195199300151961
:100180009200951891001518900014280C308C00DE
:100190000B1DC8288B018C0BC82808009601160877
:1001A0009620C620C620960A16080A3A031DCF28B4
:0201B000CE2857
:02400E00F93F78
:00000001FF
